S31508000000280C002061010008870100088901000802
S3150800001000000000000000000000000000000000D2
S315080000200000000000000000000000008B0100082E
S3150800003000000000000000008D0100088F01000884
S31508000040910100089101000891010008910100083A
S31508000050910100089101000891010008910100082A
S31508000060910100089101000891010008910100081A
S31508000070910100089101000891010008910100080A
S3150800008091010008910100089101000891010008FA
S3150800009091010008910100089101000891010008EA
S315080000A091010008910100089101000891010008DA
S315080000B091010008910100089101000800F002F87A
S315080000C000F03EF80CA030C8083824182D18A246AF
S315080000D0671EAB4654465D46AC4201D100F030F887
S315080000E07E460F3E0FCCB6460126334200D0FB1A99
S315080000F0A246AB4633431847041D0000241D0000E2
S31508000100103A02D378C878C1FAD8520701D330C852
S3150800011030C101D504680C60704700000023002434
S3150800012000250026103A01D378C1FBD8520700D320
S3150800013030C100D50B6070471FB51FBD10B510BD87
S3150800014000F0F8F81146FFF7F7FF01F0C5FD00F0DB
S3150800015010F903B4FFF7F2FF03BC00F017F900002B
S315080001600F4880F308880F480168090E0E4A914225
S3150800017005D10E480E4901600E480F4901600F4827
S3150800018080470F480047FEE7FEE7FEE7FEE7FEE783
S31508000190FEE700000B480C490C4A0D4B704700005F
S315080001A0280C0020040000001F0000001810024060
S315080001B0010000000000014000000000651500086D
S315080001C0BD00000828060020280C0020280800206A
S315080001D028080020002203098B422CD3030A8B42ED
S315080001E011D300239C464EE003460B433CD4002221
S315080001F043088B4231D303098B421CD3030A8B4233
S3150800020001D394463FE0C3098B4201D3CB01C01A00
S31508000210524183098B4201D38B01C01A52414309CB
S315080002208B4201D34B01C01A524103098B4201D3B9
S315080002300B01C01A5241C3088B4201D3CB00C01A26
S31508000240524183088B4201D38B00C01A524143089E
S315080002508B4201D34B00C01A5241411A00D20146C3
S315080002605241104670475DE0CA0F00D0494203105C
S3150800027000D34042534000229C4603098B422DD3AB
S31508000280030A8B4212D3FC22890112BA030A8B4253
S315080002900CD3890192118B4208D3890192118B42A2
S315080002A004D389013AD0921100E08909C3098B4227
S315080002B001D3CB01C01A524183098B4201D38B016A
S315080002C0C01A524143098B4201D34B01C01A52410D
S315080002D003098B4201D30B01C01A5241C3088B4252
S315080002E001D3CB00C01A524183088B4201D38B003D
S315080002F0C01A5241D9D243088B4201D34B00C01AC7
S315080003005241411A00D20146634652415B101046DB
S3150800031001D34042002B00D54942704763465B1023
S3150800032000D3404201B50020C046C04602BD704712
S3150800033070477047754600F025F8AE4605006946D1
S315080003405346C008C000854618B020B5FFF722FFFF
S3150800035060BC00274908B6460026C0C5C0C5C0C54A
S31508000360C0C5C0C5C0C5C0C5C0C5403D49008D464D
S31508000370704710B50446C046C0462046FFF7E9FE5A
S3150800038010BD000000487047C80500200149182024
S31508000390ABBEFEE726000200704700F09AFBFCE7BA
S315080003A010B500F051FB01280ED0084C2078012822
S315080003B00AD101F007F96168FF31F531884203D3A4
S315080003C00020207000F0A6FB10BD0000D800002019
S315080003D010B5044C0120207001F0F4F86060FFF7B6
S315080003E0DFFF10BDD800002010B500F07AFB00F042
S315080003F067FB01F0EFF800F04FFF00F015FBFFF781
S31508000400E7FF10BD10B500F064FB01F0FDF800F041
S315080004101FFBFFF7C5FF10BD10B501214C0620468E
S3150800042000F062FF0021204600F05EFF10BD0000CC
S3150800043010B5827A0123194691402A4A14681C434A
S315080004401460D3698B43D361037B002B12D1D36825
S315080004508B43D360C38844881B042343847AE4000F
S31508000460A4182364838804881B042343847AE4003D
S31508000470A4186364037B012B12D1D3680B43D360A2
S31508000480038844881B042343847AE400A41823645D
S315080004908388C4881B042343847AE400A41863640D
S315080004A0C37A002B06D053680B4353600389002B8D
S315080004B004D006E053688B435360F7E753698B43D0
S315080004C053610389012B02D153690B435361407B66
S315080004D0012802D1D0690843D0611068400840005D
S315080004E0106010BD0066004010B5002203680224A3
S315080004F0A34303600368012423430360384B00E0E9
S31508000500521C4468E40701D19A42F9D14268D207DD
S315080005103ED08C798022012C3CD004689443046038
S31508000520CC794022012C39D00468944304600C7AB3
S315080005302022012C36D00468944304604C7A102299
S31508000540012C33D00468944304608C7A0822012C69
S3150800055030D0046894430460CC7A0422012C2DD050
S315080005600468944304608A78CC7892072406224368
S315080005700C79240422434C79098824052243491E10
S315080005800A43C261016849084900016000211AE06E
S31508000590002010BD046814430460C1E704681443CE
S315080005A00460C4E7046814430460C7E70468144396
S315080005B00460CAE7046814430460CDE7046814437A
S315080005C00460D0E7491C4268D20701D09942F9D1A4
S315080005D04068C00701D0002010BD012010BD0000F2
S315080005E0FFFFFF0002460020002905D0012902D19D
S315080005F010698007800F7047D0688007800F7047A2
S3150800060030B50B011B18FF3381331C6B04252C40B6
S315080006101472002C2AD01C6BE40854601C6B02254B
S315080006202C4054725C6B2407240F94725C6B240A6A
S31508000630D4749C6BD4729C6B240A14739C6B240C24
S3150800064054739C6B240E9473DC6BD473DC6B240A92
S315080006501474DC6B240C5474DB6B1B0E937420220D
S31508000660002907D001691143016130BD1C6B640D77
S315080006701460D3E7C1681143C16030BD00218171A0
S31508000680C171017241728172C1728170C170032198
S3150800069001710221417101210180704730B502467E
S315080006A0002093685B010AD49068000101D50120F7
S315080006B005E09068C00001D5022000E00420042867
S315080006C038D003019A18FF3281321368DB07DB0F33
S315080006D013600B7A002B2ED014684D681C434B7A96
S315080006E0ED002B431C4314608B7A1B071B0F8B7280
S315080006F053681B091B01536053688C7A2343536064
S315080007008C7BCB7A240623434C7B0D7B24042D0259
S315080007102C43234393608C7CCB7B240623434C7C5D
S31508000720097C240409020C432343D360116801237E
S315080007301943116030BD13684C7A23430C8864054D
S3150800074023431360D0E700000022002904D00129C2
S3150800075006D002290BD107E082681948024006E054
S3150800076082681848024002E0826817480240174922
S31508000770501A8A421CD007DC002A15D014481018D3
S3150800078014D002280DD117E0FF38FF38023815D0EB
S31508000790104940180ED001214904884201D1012090
S315080007A000E00020C0B270470220FBE70020F9E70E
S315080007B00020F7E70020F5E70120F3E70120F1E73D
S315080007C003000004000300080000031000010008ED
S315080007D0FFFFFFFB0003FFF7F7B58CB0174601A82C
S315080007E000F09EFD03980B900024124E6500A9198F
S315080007F0705D497841180C98491C41430B98FFF7DE
S31508000800E9FC00290FD10D9980B208800A49401EDB
S31508000810884208D86000305C3870A819407878702B
S3150800082001200FB0F0BD641CE4B2122CDED3002008
S31508000830F7E70000F21C0008FF03000070B58AB055
S31508000840012502951D480068019001AA02A91C48C5
S31508000850FFF7C2FF012803D09A211AA0FFF79DFDD2
S31508000860224E3046FFF7D8FD07A8FFF707FF0024FA
S3150800087008AA9470D47009946A469477D477117943
S3150800088008AA491E11706A46507908AA401E507077
S315080008906A461089908307A93046FFF725FE6A46FF
S315080008A09475D47515769481D48114825482948271
S315080008B0557603A8FFF7BCFD0AB070BDF01C00080A
S315080008C020A107002E2E5C2E2E5C2E2E5C2E2E5C72
S315080008D0536F757263655C41524D434D305F535497
S315080008E04D333246305C63616E2E6300006400400F
S315080008F0F0B585B005460F460026002400211848A5
S31508000900FFF770FE002828D06A4600211448FFF732
S3150800091077FE6846007A1349002803D1009A8A426E
S3150800092000D10124042806D101220198D2071043D8
S31508000930884200D10124012C0FD16846807A38708C
S315080009400021684604E04218D27A6A54491CC9B2A2
S315080009506A46927A8A42F6D80126304605B0F0BD34
S31508000960006400406706000070B586B002460020A5
S315080009706B461873134B01936B465873997301AB07
S3150800098004E0145C1D18EC72401CC0B28842F8D30F
S315080009900D4D01A92846FFF781FE064600F012FE16
S315080009A00446323405E000F094F800F00BFEA0424D
S315080009B005D831462846FFF7C7FE0228F3D006B009
S315080009C070BD0000E10700000064004070470000A9
S315080009D009480078002807D0012807D0022807D040
S315080009E0032807D0402070474020704708207047EA
S315080009F00020704700207047E00000200948007872
S31508000A00002807D0012807D0022807D0032807D0D6
S31508000A1040207047402070470820704700207047E4
S31508000A2000207047E000002010B501F0A9F8FFF794
S31508000A3005FF044C0120207000F072FE0020207093
S31508000A4010BD0000E000002010B501F0A7F810BDA9
S31508000A5038B569460C48FFF74BFF0C4C012805D101
S31508000A60207068460178084801F0A2F869460648E9
S31508000A7000F088FE012806D100202070684601781B
S31508000A80014801F095F838BDF0000020E00000208C
S31508000A9070B505460C46094E3078012803D1E1B2F7
S31508000AA02846FFF761FF3078002803D1E1B22846CF
S31508000AB000F0CEFE01F0E6F870BD0000E000002070
S31508000AC010B500F001F810BD10B5642000F0ACFBBD
S31508000AD010BD10B500F001F810BD10B500F0AAFB66
S31508000AE010BD10B500F001F810BD72B6704762B6B9
S31508000AF0704770B505460C46164605E020782870FE
S31508000B00641C6D1CFFF7E5FF3046761EB6B200285A
S31508000B10F4D170BD10B500F0C3FB00281CD000F05E
S31508000B201DF8002818D0FFF751FF00F067FD0121D6
S31508000B30084600F0E7FB00F0ABFB01460120C022A7
S31508000B404007FFF7D6FF032000F0B4FC00F0A0FB37
S31508000B504468FFF7CCFFA04710BD000010B500F0B1
S31508000B605BFB01214903044800F0E0FA002801D0A4
S31508000B70012010BD002010BD000800480149C860CA
S31508000B807047000000200240F0B506460B273F04D8
S31508000B90384600F06DF804280FD1084C2069022564
S31508000BA02843206166612069402108432061384650
S31508000BB000F05EF82169A9432161F0BD00200240DA
S31508000BC004200849CA68D20701D001207047CA68BC
S31508000BD0D20601D502207047C9684907FBD503200C
S31508000BE07047000000200240024801698022114334
S31508000BF00161704700200240F8B505460E46002000
S31508000C0000900B273F04384600F032F804280ED12E
S31508000C100E4C20690121084320612E80384600F0D9
S31508000C2027F8042804D02169490849002161F8BD3C
S31508000C30AD1C00950098310C0180384600F018F874
S31508000C402169490849002161F8BD000000200240D9
S31508000C5004480169090603D503494160034941600F
S31508000C60704700000020024023016745AB89EFCD9D
S31508000C7000B50346FFF7A4FF02E0FFF7A1FF5B1EDE
S31508000C80012801D1002BF8D1002B00D1052000BD89
S31508000C90FEB504460D4616461F46680A40020090F1
S31508000CA02068401C05D12046009900F017F9002855
S31508000CB02CD021680098814206D02046009900F081
S31508000CC01FF90446002C23D02068281A05192D1D63
S31508000CD00098FF30FF3002300190FFF7FAFE281B1C
S31508000CE00121001F4902884207D32046019900F0D6
S31508000CF007F90446002C0DD0251D3078761C28707F
S31508000D006D1C7F1E002FE8D10120FEBD0020FEBD10
S31508000D100020FEBD0020FEBD10B50C480068401C32
S31508000D2004D00A4800F060F900280AD0084800688C
S31508000D30401C04D0064800F057F9002803D00120CB
S31508000D4010BD002010BD002010BD0000800300204B
S31508000D507C01002070B505460C460D48411B601EF7
S31508000D60814201D2002070BD284600F055F806469B
S31508000D702819401E00F050F80146FF2E05D0FF291D
S31508000D8003D0304600F006F870BD002070BD0000A4
S31508000D90FFFF030870B505460C46A54201D9002099
S31508000DA070BD042D01D3162C01D9002070BDFFF7A4
S31508000DB04FFF3420FFF7E2FEFFF702FF012812D0AB
S31508000DC0284600F047F80546204600F043F8064650
S31508000DD0204600F059F83018401E401B401C4001C0
S31508000DE0060C002411E0FFF7FFFE002070BDFFF798
S31508000DF070FEE0024019FFF7C7FE042803D0FFF78C
S31508000E00F3FE002070BD641CA4B2B442EFD3FFF712
S31508000E10EBFE012070BD000070B5054600240C4E9F
S31508000E20FFF757FE21460C2041437058A84209D8BF
S31508000E30891949684018A84204D90C204443A019C6
S31508000E40007A70BD641CE4B2132CE9D3FF2070BD90
S31508000E50181D000870B5064600240A4DFFF739FE2E
S31508000E600C2060434019007AB04203D10C20444359
S31508000E70285970BD641CE4B2132CEFD30020C0437C
S31508000E8070BD0000181D000870B5064600240A4DFE
S31508000E90FFF71FFE0C2060434019007AB04204D1C8
S31508000EA00C2044436019406870BD641CE4B2132CDE
S31508000EB0EED3002070BD0000181D000800487047DA
S31508000EC00020000800200349C04308600249086062
S31508000ED0704700007C0100208003002010B5CA0579
S31508000EE001D0002010BD02688A4201D1012010BD40
S31508000EF002C001225202FFF7FCFD012010BD0000CE
S31508000F0070B504460D460E48844201D10D4C0AE0E0
S31508000F100D48854202D10A4C054604E0204600F0F9
S31508000F2063F8002807D029462046FFF7D7FF002890
S31508000F3003D0204670BD002070BD002070BD0000A3
S31508000F40800300207C010020002000080B4801686F
S31508000F504268511882685118C268511802695118B6
S31508000F6042695118806940180449C031096808184F
S31508000F70002801D000207047012070470020000893
S31508000F8070B504460D4616461348011B681E814275
S31508000F9001D2002070BD2046FFF73EFFFF2811D082
S31508000FA06019401EFFF738FFFF280BD0600A400281
S31508000FB00A49884208D12B46324621460848FFF797
S31508000FC067FE70BD002070BD2B4632462146054897
S31508000FD0FFF75EFE70BD0000FFFF03080020000853
S31508000FE0800300207C010020F8B50546012000900A
S31508000FF02868FFF711FFFF2819D0FFF729FE3420CC
S31508001000FFF7BCFDFFF7DCFD012812D00024286895
S31508001010A100461848194768FFF75BFD3946304670
S31508001020FFF7EAFD042808D0002000900EE0002013
S31508001030F8BDFFF7D9FD0020F8BD3068B84202D0E8
S315080010400020009002E0641C802CE0D3FFF7CCFD62
S315080010500098F8BD08B5002000900E480168491CA4
S3150800106015D0416882685118C2685118026951182A
S315080010704269511882695118C0694018C043401C1A
S3150800108000906A4604210448FFF77AFF08BD01204C
S3150800109008BD000080030020C0200008F0B500222B
S315080010A00325012393400C681C409C422AD10C79E5
S315080010B0012C01D0022C12D1876854002E46A64076
S315080010C0B74387604E79A64084682643866084883D
S315080010D09C43848084888B7993401C43848006686B
S315080010E053002C469C40A64306600E7907689E402E
S315080010F03E430660C668A643C660CC799C40C36872
S315080011001C43C460521C102ACBD3F0BD10B54B0744
S31508001110DB0E9A40C90889000818016A0F249C400A
S31508001120A1430162016A1143016210BD0246002013
S31508001130128A0A4200D001207047018570478161F2
S3150800114070470000FEB501214F04384600F0B0F89C
S315080011502020009001256846057100248471032625
S315080011604671C47109206946C006FFF797FF092032
S315080011702021C006FFF7E1FF0121C80400F098F816
S3150800118068460471C4716803009069462048FFF7F1
S3150800119085FF0121384600F099F80121384600F00C
S315080011A087F8092001220221C006FFF7AFFF0920B0
S315080011B001220321C006FFF7A9FF0C20009068460C
S315080011C04671022707718471C57109206946C006F0
S315080011D0FFF764FF0121480600F078F8012188042A
S315080011E000F066F8042208210A48FFF78FFF042258
S315080011F009210848FFF78AFF300200906846077100
S3150800120046718471C57169460248FFF747FFFEBDFE
S31508001210000800480004004810B509202021C0062F
S31508001220FFF78BFF10BD000001494880704700009A
S31508001230D000002010B500F0C5F90D4C6168884251
S315080012400ED321780920C00600290AD00021217072
S315080012502021FFF772FF00F0B5F961884018606039
S3150800126010BD012121702021FFF769FFF3E7000077
S31508001270D000002010B5FFF7EDFE002802D0FFF7DA
S315080012804BFD10BD002010BD10B5FFF763FD10BD66
S3150800129010B5FFF713FE10BD10B5FFF713FE10BD0E
S315080012A010B5FFF753FE10BD10B5FFF769FE10BD68
S315080012B0054A002903D051690143516170475169B4
S315080012C0814351617047000000100240054A002919
S315080012D003D0D1690143D1617047D1698143D16196
S315080012E07047000000100240054A002903D0116922
S315080012F0014311617047116981431161704700000C
S3150800130000100240054A002903D091690143916102
S31508001310704791698143916170470000001002404F
S31508001320F8B5044600215C4E70680C2210405B4DEF
S31508001330002820D0042820D0082820D00C2839D00E
S3150800134025607068F02210400009554B1F5C206824
S315080013500246FA4094466260726807273F023A409E
S31508001360120A9B5C6246DA40A260336BDB0524D422
S315080013704C4BE36029E02560E3E72560E1E7716807
S315080013800F208004014070680322D20310408F0C9E
S31508001390BF1C00280AD0F06A0107090F491C284615
S315080013A0FEF718FF784301462160CAE73E483946EA
S315080013B04143F9E73D482060C3E773685B0402D4FC
S315080013C05308E36001E09308E360336B5F06384B2C
S315080013D003D4374F1237276100E02361376BFF06C6
S315080013E001D4656100E06061376BBF070ED0376BCB
S315080013F0BF07BF0F012F0BD0376BBF07BF0F022FD9
S3150800140008D0376BFF43BF0706D006E0A26104E0A9
S31508001410A06102E0A36100E0A561376BBF03BF0FBF
S315080014200FD0376BBF03BF0F012F0CD0376BBF032D
S31508001430BF0F022F09D0376BBF03BF0F032F06D08C
S3150800144006E0E26104E0E06102E0E36100E0E561F4
S31508001450376B3F03BF0F0FD0326B1203920F012A6F
S315080014600CD0306B0003800F022809D0306B0003C4
S31508001470800F032806D006E0226204E0206202E01C
S31508001480236200E02562306B000602D407486062DA
S31508001490F8BD6162F8BD00000010024000127A0033
S315080014A0C0000020809FD50000093D00006CDC02CA
S315080014B000800000034A1168890889000143116009
S315080014C070470000000001401CB5002301930093FB
S315080014D022480168012212041143016051000524C3
S315080014E0240302680A400092019A521C0192009A4B
S315080014F0002A02D1019AA242F3D10168890302D5D2
S315080015000121009100E000930099012925D1144991
S3150800151011220A60416841604168416041687F2242
S31508001520D20391434160416811221204114341607C
S315080015300168012212061143016001688901FCD580
S315080015404168890889004160416802221143416067
S3150800155041680907890F0229FAD11CBD001002400B
S315080015600020024010B514480168012211430160A9
S315080015704168124A114041600168114A11400160F0
S315080015800168012292049143016041683F221204D6
S3150800159091434160C16A09090901C162016BFF22D1
S315080015A0543291430163416B490849004163002164
S315080015B08160FFF789FF10BD001002400CB8FF08D4
S315080015C0FFFFF6FE00B500F01FF80148006800BDF1
S315080015D0E400002000B500F011F80648044941610E
S315080015E000218161052202610348016000BD0000F7
S315080015F07FBB000000E000E0E40000200149002075
S315080016000861704700E000E004480069C00303D59C
S3150800161003480168491C01607047000000E000E0CB
S31508001620E4000020002904D001680122114301606A
S315080016307047016849084900016070470246002062
S31508001640D2690A4200D001207047000030B58BB03D
S3150800165004460D4620684008400020606068032163
S3150800166009038843A9680143616020681E49084048
S31508001670EA68696811432A69024311432160A06830
S3150800168003210902884369690143A16001A8FFF79C
S3150800169047FE1648844201D107980AE01448844256
S315080016A001D1089805E01348844201D1099800E061
S315080016B003982168090404D540002968FEF78AFDC5
S315080016C002E02968FEF786FD2A6852088A4200D891
S315080016D0401C2168090404D50107490F064A104031
S315080016E00843A0810BB030BDF3E9FFFF0038014085
S315080016F00044004000480040F0FF000082680123D3
S315080017001B039A43826082680A4382607047808C12
S31508001710C005C00D7047C905C90D01857047000091
S3150800172010B586B0E12000020090002001900290DA
S31508001730039005900C200490074C69462046FFF755
S3150800174085FFA1142046FFF7D9FF01212046FFF7A0
S3150800175069FF06B010BD00000044004070B504469D
S31508001760074D20212846FFF769FF012801D00020F0
S3150800177070BD2846FFF7CBFF2070012070BD000022
S3150800178000440040F3B581B00F461B4C0025607835
S315080017901A4E00280FD020783018401CFFF7DEFFBD
S315080017A0012818D0FFF70EFF61686431884200D916
S315080017B065700020FEBD1148FFF7D0FF0128F8D15B
S315080017C03078401E3F28F4D8FFF7FCFE606025708D
S315080017D001206070EDE72078401CC2B22270307894
S315080017E09042E6D1711C0198FFF783F9657020785D
S315080017F038700120FEBD0000E800002084050020A6
S3150800180070B504460125114E80213046FFF716FFB4
S31508001810002808D021463046FFF77DFFFFF7D2FEA5
S3150800182004460A3409E0002070BDFFF752F9FFF7B5
S31508001830C9FEA04201D9002505E080213046FFF700
S31508001840FDFE0028F1D0284670BD00000044004087
S3150800185070B506460D46402D03D982210EA0FEF727
S315080018609CFD2846FFF7CCFF012803D086210AA055
S31508001870FEF793FD00240CE0FFF72BF9305DFFF728
S31508001880BFFF012803D08F2103A0FEF786FD641C45
S31508001890A4B2AC42F0D370BD2E2E5C2E2E5C2E2E3A
S315080018A05C2E2E5C536F757263655C41524D434DD9
S315080018B0305F53544D333246305C756172742E6313
S315080018C00000000010B5084CFF21E1704168E21DD8
S315080018D0A06C00F043F9207100206071A071082106
S315080018E020464030818010BD3001002070B500F0E0
S315080018F0CFF90E4C01252570FF20E070002110203D
S3150800190020716171FFF764F8A071FFF777F8E0714D
S31508001910FFF774F8000A20726572A572204608213E
S3150800192040308180FFF7B8FC70BD00003001002010
S3150800193010B5064C0020207000F0AAF9FF20E070D0
S31508001940012120464030818010BD00003001002072
S315080019500748FF21C170074981640021017141715F
S3150800196081710721C01C416008213D308180704784
S3150800197030010020E61C00080648FF21C17000213E
S315080019800171427842718171C1710172062140303C
S31508001990818070473001002070B50446FFF718F8BB
S315080019A06178801E884203DA222000F077F970BD3C
S315080019B0104DFF20E870012128464030818061786B
S315080019C000290AD0A21CA86CFFF76EFC00280CD0D0
S315080019D06178A86C4018A86470BDFFF74BFC002816
S315080019E0FAD1312000F05AF970BD312000F056F9CD
S315080019F070BD00003001002010B5094C4168A06C8C
S31508001A00FFF742FC002806D0FF20E070012120469F
S31508001A104030818010BD312000F040F910BD000033
S31508001A203001002070B50546FEF7D2FF0C4C411E6A
S31508001A306A1CA06CFFF738FC00280CD0FF20E07069
S31508001A40FEF7C6FFA16C401E4018A064012120467F
S31508001A504030818070BD312000F020F970BD000053
S31508001A603001002010B5312000F018F910BD000033
S31508001A7010B5FFF74FF80449FF20C8700248012146
S31508001A804030818010BD00003001002070B5084C40
S31508001A90FF20E070002525716571FEF799FFA0719A
S31508001AA0E57125726572072120464030818070BD38
S31508001AB0300100200449FF22CA7040688864024841
S31508001AC001214030818070473001002070B50446FE
S31508001AD0FEF77EFF6178401E884203DA222000F076
S31508001AE0DDF870BD094D6168A9646278281DFFF7A5
S31508001AF000F8FF20E8706178A86C4018A864607840
S31508001B002946401C4031888070BD00003001002005
S31508001B1010B5002000F0C2F810BD000070B50546EB
S31508001B20FEF756FF6A78401E904203DA222000F03C
S31508001B30B5F870BD084C201DA16CFEF7DAFFFF2032
S31508001B40E0706978A06C4018A06468782146401C4B
S31508001B504031888070BD000030010020F8B5044689
S31508001B600E461746002505E02078641C4019C5B2C4
S31508001B70FEF7AFFF761E701CF6D13D600120F8BD5A
S31508001B80054A00201070906411464031C87088805C
S31508001B9090705070704700003001002003480078AC
S31508001BA0002801D00120704700207047300100202E
S31508001BB070B50178324CFF290FD02278012A5ED100
S31508001BC0F42921D013DCD02936D009DCC92930D034
S31508001BD0CC293DD0CF293ED137E0FFF787FE3DE03F
S31508001BE0D1292FD0D2292AD0F32934D112E0F539B8
S31508001BF00B0000F064F80A060C3030301230151865
S31508001C001B30FFF78BFF29E0FFF760FF26E0FFF7A1
S31508001C1051FF23E0FFF756FE20E0FFF799FE1DE08F
S31508001C20FFF776FF1AE0FFF7A7FE17E0FFF780FE3B
S31508001C3014E0FFF7F7FE11E0FFF7AEFE0EE0FFF740
S31508001C4025FF0BE0FFF7D8FE08E0FFF711FF05E0D8
S31508001C50FFF708FF02E0202000F020F8084D403585
S31508001C60E878012802D1102000F018F80421695EEE
S31508001C70002904DD0120E870E01C00F01BF870BDA7
S31508001C803001002001480021C17070477001002012
S31508001C900149002048707047300100200449FE229F
S31508001CA0CA700871024802214030818070470000DE
S31508001CB03001002010B589B2FEF7EAFE10BD30B437
S31508001CC07446641E2578641CAB4200D21D46635DCB
S31508001CD05B00E31830BC1847FFF734FAFEF784FBBD
S31508001CE0FEF790FBFCE74F70656E424C540000000F
S31508001CF0010105020602060307030803090309048E
S31508001D000A040B040C040C050D050E050F050F0639
S31508001D101006100710080000002000080008000040
S31508001D200400000000280008000800000500000064
S31508001D30003000080008000006000000003800080F
S31508001D400008000007000000004000080008000026
S31508001D50080000000048000800080000090000000C
S31508001D6000500008000800000A000000005800089B
S31508001D70000800000B0000000060000800080000D2
S31508001D800C00000000680008000800000D000000B4
S31508001D9000700008000800000E0000000078000827
S31508001DA0000800000F000000008000080080000006
S31508001DB0100000000000010800800000110000006B
S31508001DC000800108008000001200000000000208E0
S31508001DD00080000013000000008002080080000058
S31508001DE01400000000000308008000001500000031
S31508001DF00080030800800000160000001C1E000872
S31508001E00C000002030000000000100084C1E000839
S31508001E10F0000020380B00001C010008000000003C
S31508001E200102030401020304060708090000000072
S31508001E300000000000000000000000000400000090
S31108001E4000000000000000000000000088
S705080000BD35
